:100000008A110A120528000009000730990083169A
:10001000051085100511851605168312E830A0001D
:100020000330A10046219920851A1B28051E192896
:1000300044201F3083051F3083055A30A000A101E2
:1000400046213008013EB00030080A3C031D2C2830
:10005000B0013108013EB1001F30830531083C3C3E
:10006000031D3628B1013208013EB2001F3083055E
:1000700032080F3C031D40289920B201B101B001A4
:100080001F3083051428432805140130AF00B00148
:10009000B101B201051E87285A30A000A1014621F6
:1000A0003008013EB00030080A3C031D5B28B00157
:1000B0003108013EB1001F30830531083C3C031D6F
:1000C0006528B1013208013EB2001F3083052F08B8
:1000D000013C031D77283208023C031D75280510DA
:1000E0000E30B2003230B100AF011F3083051F3037
:1000F000830532080F3C031D842899200514342100
:100100000510B201B101B0011F3083054A281F302C
:100110008305AF01C830A000A1014621DE203230A6
:10012000A000A101462105100E30B2002D30B10013
:1001300008000514F430A0000130A1004621FC2085
:10014000C520EE20D220EE20E220EE20C320EE20BB
:10015000CA20FC20C020EE20D920EE20C320EE20B3
:10016000C520EE20C520EE20C020EE20D620EE20B7
:10017000C320EE20CE20EE20C020FC200510080079
:10018000122123210800122108001221232112210B
:1001900012210800232123212321080023211221D9
:1001A00012210800122112212321080023211221EB
:1001B00008001221122112212321080023211221DB
:1001C00023210800232123211221122112210800BA
:1001D00005113C30A000A1014621080005113C306A
:1001E000A000A10146213C30A000A10146213C30E5
:1001F000A000A1014621080005113C30A000A1018A
:1002000046213C30A000A10146213C30A000A101C4
:1002100046213C30A000A10146213C30A000A101B4
:10022000462108000515053084000230AA00F3308D
:10023000A0000130A1003C30A2000030A3008121C9
:100240000511E82008000515053084000230AA00D9
:10025000F330A0000130A100F030A2000030A30074
:1002600081210511E82008000515053084000230C1
:10027000AA00F330A0000130A100DC30A20005305C
:10028000A30081210511E82008004529A0080319D1
:1002900051295821A00300000000000000000000C8
:1002A0004629A108031908005821A103A0034629E3
:1002B0000C30A500A50B5A29000000001230A20046
:1002C000A20B67296921692100000000080069214B
:1002D00060290D30A400A40B6B2900000800103029
:1002E000A8020001031C013EA902031C0800782992
:1002F0000A30A8020001031C013EA902031C0800E9
:1003000078292A0880042008A8002108A9006F2164
:100310000130A202031CA3032A0980052008A800BB
:100320002108A9006F21A208031D8129A308031D2C
:040330008129080017
:02400E00C431BB
:00000001FF
